:020000020000FC
:10000000F7C991C20000000025C000004FC10000E8
:10001000000052C1000000000000000002030406BE
:10002000080C101820304060800002030406080C01
:10003000101820304080FF000406080C10182030F3
:10004000406080A0C0000D0D0403060D050D0603E1
:10005000030202004FB662FD1EC070FF1AC165FDAB
:10006000FAC00994C0919700C395C0939700C5E06A
:10007000C519B8F3D0919700CD1B98F3C8E7089441
:1000800083FDC795C4BDC52DCC2321F4C0E083FDFD
:10009000C0E8C4BD09C171FF03C09598AC98C09871
:1000A000C52D089483FDC795C4BDC09399006B7F8F
:1000B000C52DCF3F09F443C0C0919800C395C093AC
:1000C000980070FF37C082FD05C09598AC98C09825
:1000D0004FBE18957860C091A000CC2391F0C091DC
:1000E0009800CA95D091A000CD1B58F0777FC091A1
:1000F0009800D0919F00CD1B08F41CC0209298005E
:1001000019C09598AC98C098C5E0CA95F1F7C09110
:100110007500CA95C2FD09C0C1FD05C095FFAB9A27
:1001200095FD949A0EC0AD9A0CC095FF949A95FDDA
:10013000AB9A07C09598AC98C0984FBE189520927E
:1001400099004FBE1895A5C0552021F095FF959AAE
:1001500095FDC09AAC989DC0552009F0AC9A95FFCA
:10016000C09895FD959895C0552021F095FFC09AAF
:1001700095FD959A95FF959895FDC0988AC095FF35
:10018000949895FDAB9895FFAB9895FD9498C5E034
:10019000CA95F1F7552021F095FF959A95FDC09AE3
:1001A000AC9877C095FF949895FDAB98AD98C5E055
:1001B000CA95F1F7552021F095FF959A95FDC09AC3
:1001C000AC9867C0AD9895FF949895FDAB98C5E045
:1001D000CA95F1F7552009F0AC9A95FFC09895FDA6
:1001E000959857C0AD9895FFAB9895FD9498C5E04C
:1001F000CA95F1F7552009F0AC9A95FFC09895FD86
:10020000959847C095FFAB9895FD9498AD98C5E03B
:10021000CA95F1F7552021F095FFC09A95FD959A62
:1002200095FF959895FDC09834C095FFAB9895FDC6
:10023000949895FF949895FDAB98C5E0CA95F1F711
:10024000552021F095FFC09A95FD959A95FF9598B8
:1002500095FDC0981EC082FF1CC0C0917500C2FDF4
:100260000BC0C1FD11C095FF949895FDAB9895FF0B
:10027000AB9895FD94980DC0C1FDF5CF95FF94986E
:1002800095FDAB98AD9805C0AD9895FFAB9895FDE1
:100290009498C52DC095089483FDC795C4BDC0939F
:1002A00099002092970064604FBE18954FB6C0E148
:1002B000C8BF6E7F4FBE18953FB68F7EABB7A07498
:1002C000A2118061A0E0ABBFA9B7AE7FA9BF7894AF
:1002D000A0916600AA2349F0A92FAF7151F1A09116
:1002E0006600AA95A093660024C040E050E0A0B349
:1002F00096FDA095A2FD4FEF96FFA3E096FDA2E02C
:10030000A5BFAA27A064AABF8D7FA0B396FDA09524
:10031000A2FD5FEF451749F7A0E461FDA0936600D9
:10032000A92FAF7119F0A0E4A093660040938D004F
:100330008160A0916700AA2331F0A0916700AA957F
:10034000A093670007C0A92FAF7121F08061AA2791
:10035000A064AABF80FF30C0A0918D004A2F8E7F7D
:10036000A92FAF7109F000C04093610071FF08C070
:10037000A091610050919200A51710F05093610078
:100380004091AE004430C1F4A091610040916300FF
:10039000A41B70F04091CF00A40B50F0A09163001B
:1003A000A40FA093630040F4AFEFA093630004C0D8
:1003B000A0916100A0936300A52DA03408F06860AF
:1003C000A0916000A395A093600051F0F894A9B7A4
:1003D000A160A9BF84FF02C0A0E4ABBF3FBE1895D7
:1003E00042E050916600552331F0A92FAF7119F406
:1003F0005A9550936600A0918D00A13018F020927C
:1004000090000DC02092910020929A00A09190003F
:10041000AF5FA093900018F0AFEFA0939000B09062
:1004200061005091AE00523049F466FF91F0A2E3B2
:10043000BA1678F0A0917F00A0936100533049F480
:1004400066FF39F0A2E3BA1620F0A091BA00A0939B
:100450006100509162005B1521F010F05A9501C0C7
:100460005395509362004A95D1F650919A00539556
:1004700009F45A9550939A00A0919B00AA95A093D5
:100480009B0009F046C0A1E0A0939B0045E0A0912D
:100490009C005A17F0F1A0919D005A1728F441E0F2
:1004A000A3E0A0939B0007C0A0919E005A1718F4E8
:1004B00041E040939B00D0909300C0906300DC1417
:1004C000A8F0A091AE00A430D9F066FD0FC0C09294
:1004D0009300539519F0A0919C00A0939A00A1E07D
:1004E000A0939B00ACE3A093620013C0A091930083
:1004F000A40F20F45FEF5093930002C0A0939300E9
:10050000A0919300AF3F29F4AFEFA0939100A09387
:100510009A00F894A9B7A160A9BF84FF02C0A0E423
:10052000ABBF3FBE18953FB64CB55DB58F7EABB740
:10053000A074A2118061A0E0ABBFA9B7AE7FA9BF34
:10054000789481FD26C096FFA2E096FDA3E0A5BFAA
:100550008260A0B396FDA095A2FF05C04093640001
:1005600050936500FDC096FFA3E096FDA2E0A5BFF5
:10057000AA27A064AABF8D7FA92FAF7109F4E1C09B
:1005800040E0A0B396FDA095A2FDDBC040938D0096
:10059000CEC096FFA3E096FDA2E0A5BF8D7F61FFD0
:1005A0006BC096FFA2E096FDA3E0A5BFAA27A064BA
:1005B000AABF82604093880050938900A090860073
:1005C0004A19B09087005B09BB24A2E0EA2EA22C56
:1005D000483CA0E05A0730F4A0E1BA2EE22CAAE091
:1005E000AA2E27C04836A1E05A0730F4A8E0BA2E58
:1005F000E22CAFE0AA2E1DC0403DA2E05A0730F425
:10060000A4E0BA2EE22CAEE1AA2E13C0403AA5E037
:100610005A0730F4A2E0BA2EE22CACE3AA2E09C0AD
:100620004839A8E05A0728F4A1E0BA2EE22CA8E73E
:10063000AA2EC42EA0918A00CA1AD52EA0918B0092
:10064000DA0ADD202AF4AFEFC094D094CA1ADA0A8D
:1006500020928C00CA14DE0418F4A1E0A0938C0050
:1006600040938A0050938B004091880050918900FC
:100670004093860050938700A09164004A1BA0918C
:1006800065005A0B94FD46C093FD44C092FD40C0E6
:100690005695479591FD3CC05695479590FD38C0BD
:1006A000D52EC42ED694C79461FD0CC0AC2DAC5190
:1006B000AD2DA24008F045C0DD2021F4AC2DA85C92
:1006C00008F43FC0A0E0EA2E97FD02C0E090C2000F
:1006D000AAEFEA0EF22CF21CCE18DF084FB74170D9
:1006E000442319F040E050E015C0AFEFCA16D20421
:1006F00018F04FEF50E00EC0F090A700CF9C412DB6
:10070000000C441F50E008F012C04FEF50E00FC043
:100710005695479594FF07C0552309F04FEFA42F36
:10072000A6954A0F521D4F3F520508F04FEF4093D8
:100730008D00816061FF05C0AFE1A095A923AB29C1
:100740009A2FA0E4A0936600A92FAF7119F4AAE034
:10075000A093660061FD04C0A92FAF7109F08F7EE0
:10076000A0E2A0936700A92FAF7119F4AAE0A093AB
:100770006700F894A9B7A160A9BF84FF02C0A0E4F4
:10078000ABBF3FBE189511E00AC013E008C01AE0E5
:1007900006C01EE104C014E602C018EC00C005E16A
:1007A000BB27BA95F1F70A95D9F71A95C1F70895BD
:1007B0002AE338E709C020E33CE806C02AE234EB2C
:1007C00003C025E238EC00C0652CB1E05B2E12E0DE
:1007D00095FD9F7D95FF9062BB27AD98BA95F1F787
:1007E000552009F0AC9ABA95F1F7AC98BA95F1F7A3
:1007F000AD9ABA95F1F7552021F095FF959A95FDA0
:10080000C09AB091A800BA95F1F795FF959895FD1B
:10081000C098B7E8BA95F1F71A95D1F6022FB22F22
:10082000BA95F1F70A95D9F73A9571F6AD98562C25
:100830000895221B39E0001F3A9509F40895221FFC
:10084000211B18F4210F8894F6CF0894F4CF622C62
:10085000722CB0E08894B395221F331FE0F73795D0
:1008600027958894912E802E020B130B10F4192DCE
:10087000082D10F4889401C00894661C771CBA9562
:1008800071F7172D062D0895322D11232AF43A956C
:1008900000951095031B130BF894029F712C002DEB
:1008A000129F912C802C7894780C172D921C292D56
:1008B000B4E06B2E2695179507956A94D9F73323E4
:1008C00021F000951095031B130B08950091AE00C5
:1008D000043009F474C0B0918D00B95198F0B72F6D
:1008E000B67081F466FD2BC005E09090C000B92D74
:1008F000BA9521F00AE0BA9509F002E1B0917400CE
:10090000B01BE0F066FF0AC0B0919500B093930071
:10091000BFEFB0939A00B1E0B0939B00B09161003B
:10092000B0936300209277002092780020927900A3
:1009300020927A0020927B006F7B41C0606490908F
:10094000C000B92DBA9579F4B0916200B095BB1F83
:10095000BB1F1B2FB7950B2FB12FB170B3951B2F5A
:10096000B02FBE7F25C0B92DBA95BA9581F4B0914C
:100970006200B095BB1FBB1FBB1F1B2FB7950B2F72
:10098000B12FB370B3951B2FB02FBC7F14C0B091A3
:100990006200B095BB1FBB1FBB1FBB1F1B2FB795B2
:1009A0000B2FB12FB770B395B3951B2FB02FB87F16
:1009B000B0540B2F1209009377001093780008951C
:1009C00066FF21C010917400169500917300079581
:1009D000B0917700B01B0B2FB0917800B10B1B2F9B
:1009E00028F40038BFEF1B0740F009C00F3712058D
:1009F00008F405C00FE710E002C000E81FEF009305
:100A00007C0010937D00089566FF39C000917C0042
:100A1000B09179000B0F10917D00B0917A001B1FEF
:100A200020E030917D0033230AF42A95B0917B00B9
:100A30002B1F1AF4203F40F00AC02F3008F407C0E3
:100A40000FEF1FEF2FE003C000E010E020EF309128
:100A50006300B09192003B1718F4332331F009C0C2
:100A6000B0917D00BB235AF004C0B0917D00BB2340
:100A700032F40093790010937A0020937B0008955C
:100A800066FF2FC02091CD0000917C00000F1091D7
:100A90007D00111FF9DE11232AF40038BFEF1B0778
:100AA00040F009C00F37120508F405C00FE710E049
:100AB00002C000E81FEF002352F0B0916200B01BAB
:100AC0000B2F18F0013008F00AC001E008C00095B3
:100AD0000F5FB09162000B0F08F001C00FEF0093A1
:100AE0007E00089566FF2DC02091CE0000917A000F
:100AF00010917B00C9DE11232AF40130BFEF1B07E0
:100B000040F009C00F3F120508F405C00FEF10E0D8
:100B100002C001E01FEF112352F0B0917E00B01B24
:100B20000B2F18F0013008F00AC000E008C0009553
:100B30000F5FB0917E000B0F08F001C00FEF009324
:100B4000630008950FEF677FB72FB670E9F4686010
:100B5000B0917400B83008F0677FB0917400A1F0D4
:100B60000FEF1091740065DEF894B09170000B9F48
:100B7000112D002D7894112309F00FEFB0919500FD
:100B80000B1710F40091950000939400089506D37C
:100B900074FFB2E074FDB1E0B7B9B6B1B068B0644B
:100BA000B6B9F1DD74FFB2E074FDB1E0B7B9B6B12A
:100BB000B068B064B6B9B6B1B6FDFDCF04B115B139
:100BC000B6B1BF77B6B923D324E72093A30030E0B2
:100BD0003093A400732E7694622E6694620E731E78
:100BE000262D372D0217130778F08090A300B4E765
:100BF000B80DB093A3008090A400B0E0B81DB093EE
:100C0000A400260D371DEECF8090A3009090A40085
:100C10001091A40016950091A300079516950795CD
:100C2000B091A300B00FB093A100B091A400B11F88
:100C3000B093A20023E0169507952A95E1F720913D
:100C4000AF002A9529F42092A3002092A4000AC0A4
:100C50002A9521F0800E911E2A95E1F78092A3003B
:100C60009092A40008952091AF00B6B1B6FDFBCFDD
:100C700004B115B1B6B1BF77B6B9B091A500B395BF
:100C8000B093A500B83060F12092A500B091CC00DF
:100C9000BB2321F1112329F0B091A600BF3F61F0E1
:100CA00009C0B091A6000B1739F020F4BB2321F046
:100CB000BA9502C0B395E1F300919200B093A600FB
:100CC000BC3B50F400ECBE3A38F400E8B03A20F4F3
:100CD00000E4B23908F400E0009392007F7E0895AA
:100CE000213099F00F3FB3E01B0778F4B091A300D7
:100CF0000B17B091A4001B0740F4B0919200BB23E6
:100D000059F0BA95B093920007C0B0919200BF3FDE
:100D100019F0B395B093920000919200B0916300E6
:100D2000B01B10F400916300B09193000B1750F0CA
:100D300000919300B0919300BF3F21F0B0919300D8
:100D4000B0939200502EB091A500B73009F47061B5
:100D5000089502E3F894B091D0000B9F012D000C90
:100D6000001F7894B09192000B1710F00091920040
:100D70000093610000936300502E00939500089546
:100D800020927300B8E0B093740008952091800021
:100D900030918100F8940CB51DB5200F311F3BBD7B
:100DA0002ABD6160B0E1B8BF7894209171003091A4
:100DB00072000093710010937200021B130B2091BC
:100DC000730030917400622E732EB4E08B2EB2E06B
:100DD0009B2EB0917400B43010F08A949A94B8307D
:100DE00010F08A949A94769467948A94E1F726197D
:100DF0003709992021F0169507959A94E1F7200F6D
:100E0000311F209373003093740008F00895BFEFF2
:100E1000B0937300B09374000895209182003091D4
:100E20008300F8940CB51DB5020F131F1BBD0ABD3E
:100E30006160B0E1B8BF7894089560FDFECFEDDF4A
:100E40000895B091BE0000916E00023808F0B3958D
:100E5000003A08F0B395B63008F0B5E09B2EBCE040
:100E60008B2EB0917400B33030F48394839482FF5E
:100E700002C083948394B23030F48394839482FFCD
:100E800002C08394839471FF03C0B3E09B2E822C35
:100E9000109174000091730024E0169507952A952F
:100EA000E1F70819120928F0B02FB250B12FB2099A
:100EB00010F402E010E0312F202F712E602E769476
:100EC0006794B92DB330E9F0B0FD05C0060D171DCC
:100ED000262D372D06C0000F111F0250120922E0E7
:100EE00030E0B92DB33068F0209384003093850052
:100EF00000938000109381006092820070928300C2
:100F0000089500938400109385002093800030930F
:100F100081006092820070928300089560FDFECF90
:100F200020918200220F30918300331FB72FB670BB
:100F300021F02091730030917400F8940CB51DB528
:100F4000020F131F1BBD0ABD6160B0E1B8BF7894EA
:100F5000089560612092760020E004C060612092D4
:100F6000760020E2B72FB67009F06F7E789460FDAE
:100F700005C0B0917600BB2309F0089501E063FF3E
:100F80000AC0B0917400B33008F002E0B091740070
:100F9000B63008F003E071FF01C006E060FD06C056
:100FA000B0917600BB2311F0789408951AE083FF86
:100FB0001AE0789400000000F89462FD03C014E188
:100FC00083FF14E171FF01C018E7B4B530919900B7
:100FD000B31BB10B18F3B0917600B395B0937600C4
:100FE000B5E03B2F6B2E722CB8B1B072B21709F07E
:100FF00073943A95C9F77394761488F464FFB2CF6A
:101000006F7E3CB56DB47090730080907400370DA6
:10101000681C6BBC3ABD6160B0E1B8BFA3CF64FD92
:10102000A1CF0A9509F0BACF7894089571FF0AC04C
:10103000B0916D00B395B0936D0060FD0CC020922F
:101040006D0009C060FD07C064FD05C067FD03C0F9
:10105000BF91BF9163C408952091840030918500B1
:10106000F8940CB51DB5020F131F1BBD0ABD6160BE
:10107000B0E1B8BF78940895EFDF00E063FF03C0EC
:1010800064FF01C001E0F89410916E00B7E01B9F6F
:10109000212D102D7894200F2695179526951795BC
:1010A0002695179510936E00183718F4B8E7B0938B
:1010B0006E0000916E00B0916F000B1720F060621F
:1010C0009598AC98C09860FDFECF0895F8949498D8
:1010D000AD98AB9882FF07C0E2E0F1E073FF03C078
:1010E000B5E0BA95F1F795FF949A95FDAB9AB2E009
:1010F000B093750089C0F89495FFC09895FD9598B8
:1011000082FF0DC0E2EFF0E073FF0BC0AD9895FFDA
:10111000AB9895FD9498B5E0BA95F1F702C0ECEA6A
:10112000F0E062FF03C0552009F0AC9AB3E0B09341
:1011300075006AC0F8949498AD98AB9882FF07C088
:10114000E2EEF0E073FF03C0B5E0BA95F1F795FF6A
:10115000AB9A95FD949AB4E0B093750055C0F8949D
:10116000AC9882FF0DC0E2EDF0E073FF0BC095FF7D
:10117000949895FDAB98AD98B5E0BA95F1F702C09B
:10118000E4EAF0E062FF06C0552021F095FF959A51
:1011900095FDC09AB5E0B093750036C0F894949868
:1011A000AD98AB9882FF07C0EFEBF0E073FF03C090
:1011B000B5E0BA95F1F7AD9AB6E0B093750024C0EA
:1011C000F89495FF959895FDC09882FF10C0E5E1D1
:1011D000F1E073FF0EC095FF949895FDAB9895FFD5
:1011E000AB9895FD9498B5E0BA95F1F702C0E4EBA1
:1011F000F0E062FF06C0552021F095FFC09A95FDF2
:10120000959AB1E0B09375006F7D7894089523EAC4
:1012100030E0F9019598AC98C0989498AD98AB9847
:101220006B7F0895ACEAB0E007E00D9307E00D9303
:1012300001E00D9304E00D930FEF0D930D9309E082
:101240000D9302E00D9301E00D9301E00D93A8EBE7
:10125000B0E001E00D9300E00D9304EB0D930FEF70
:101260000D930D930D9303E00D9301E00D9301E0B9
:101270000D930FEF0D9305E20D9300ED0D9308E72D
:101280000D9308EC0D9304E00D930DE00D9301E038
:101290000D9300E00D930AE70D930AE00D9301E032
:1012A0000D9308952091BF0009E011E0223011F460
:1012B00005E011E0233011F405E012E0243011F4D0
:1012C00005E013E0253011F409E017E0263011F4B1
:1012D00000E010E000939F001093A0002091B30065
:1012E0008B7F233009F48460777F233009F47860A2
:1012F000B091B4009F7DB1FD90629F7BB091B5002D
:10130000B1FD9064B22FB23011F0886001C0877FC8
:101310000895ECE1F0E00091AC000A95E00FF21DB9
:10132000B491B093CD000091AD000A95E00FF21D8D
:10133000B491B093CE006BDF0895EAE2F0E0009143
:10134000C7000A95E00FF21DB491B093CF005FDFA4
:101350000895E8E3F0E00091B2000A95E00FF21D75
:10136000B491B093D00053DF08950091CB000023D7
:1013700009F40395013108F001E1B02FB00FB00F6F
:10138000B0939C001B2FB10FB10FB00FB0939D0015
:10139000B10FB00FB00FB0939E000895B091C80088
:1013A0000FEF1CE0B23011F400EA1AE0B33011F490
:1013B00002E815E000936F001093700008950895FF
:1013C0002091C2003091C30097FF02C020E03FEFA0
:1013D000B32FB21B6B2EB25810F4B2E86B2E00E0A4
:1013E0000395609EB12DB058D8F30093A7000895DF
:1013F000F894E3E0F0E0B9E0B7BFB491B078C1F39E
:10140000F894A895B1B5B861B1BDB0E0B1BDB4E094
:10141000BEBFBFE5BDBFFBDEB0E0B8BBB1E1B7BB4F
:10142000B0E0B5BBB8E3B4BBB0E0B2BBB0E3B1BBB6
:101430002224A0E0B0E02D92AA31E9F7A0E6B0E0C6
:101440000FEF2D920A95E9F7EDDE8DD22BDF61DFEC
:1014500074DF7FDF8ADFA2DFB2DFB2DF0091C4007A
:101460000093A800D4DEB2E0B3BFB2E0BEBDB2E0EC
:10147000B5BDF89492D99CD98CD99DD98AD99ED9D9
:1014800088D908D38AD989D986D9B1E5B8BFB9BF77
:10149000B0B7B860B0BFB6B1B460B6B974D978941B
:1014A00076DBB0E4BBBFBB27B064BABF8D7F75D914
:1014B000B1E0B0936900626025E0B0918C00BB237D
:1014C00009F425E062D9B0918D00B230A8F3B92FAC
:1014D000BF7100918F0000938E00B0938F00B01702
:1014E00059F72A9551F76D7F96FFB3E096FDB2E06C
:1014F000B5BFBB27B064BABF8D7F4DD946D902E0D6
:10150000B92FBF7109F400E0B0918D00B017B0F3AE
:10151000F8944ED94DD94CD978943FD920927F0078
:1015200034D9B091B800B13008F46CC0B091690002
:10153000B13008F467C0B92FBF71C1F0B0918D0010
:10154000BF3F08F45FC0F8943CD9789424D9B09197
:101550008D00B130C0F7F8942BD919D929D97894D6
:101560001AD9B0918D00BF3FB0F3C6C2B8E09B2E30
:101570009068F89425DF78940ED9F8949F7720DF4F
:1015800080908D00B0918D00BF37789408F442C0F0
:10159000FAD8F89416D978949A9451F7B82DB55092
:1015A000B093C300FAD8F8940BD279D27894BAE009
:1015B0009B2E9068F89404DF7894EDD8F8949F7788
:1015C000FFDE80908D00B0918D00BF37789478F762
:1015D000DAD8F894EDD8DBD8EBD878949A9449F718
:1015E000B82DBB5FB093C200D8D8F894E9D166D2C9
:1015F0007894D1D8F894E4DE7894B0918D00BF3F10
:10160000C0F37AC200918D00B0917F000B1710F0EB
:1016100000937F00C0D801E0B091B400B35009F44A
:1016200005E0B0918D00B01708F07ACFF894C9D8D2
:10163000C8D8C7D87894B1D82092690020926A009F
:1016400020926B00B0916A00B395B0936A00BF3FDF
:1016500069F5B0916B00B395B0936B00B091C60083
:1016600009E1BA9559F002E3BA9541F00DE7BA9550
:1016700029F00AEFBA9511F020926B00B0916B003F
:10168000B017A0F0B0916B00BA95B0936B00B4EBBB
:10169000B0936A00B091C500B093A800F89491D8B7
:1016A0007894B091C400B093A80075D870D8B09168
:1016B0006600BB2321F4B92FBF7109F4FCCEB091B1
:1016C0008D00B63008F4BECF66D8B0916600BB235B
:1016D00009F4F1CEF8949BDD209261002092620023
:1016E00020926300522C7894B091B100B093960090
:1016F00020927700209278002092790020927A0040
:1017000020927B002092A50060E070E020926E00A5
:1017100037DBB8E0B093A500706135D874FFB2E054
:1017200074FDB1E0B7B9B6B1B068B064B6B9B6B1DE
:10173000B6FDFDCF04B115B1B6B1BF77B6B911236F
:1017400009F00FEF0093A6008EDAB8E0B093A50081
:1017500070618090B300B2E0B093B300A3DD8092DB
:10176000B300F894BFEFB0939200F3DAB091610048
:10177000B0939200B0939300B09394007894B1E04A
:10178000B0936100B09363005B2EB0939B00B09167
:101790009100B0939A007160726020926D00FEDC3F
:1017A0000FDDF4DAEDDA4DDB04C07CDD2092A5001C
:1017B0007F7E95FFB6E095FDB0E0B7B9CFDB36DCB4
:1017C0004BDC84D859DC82DCE1DA37DB3ADBA6DBA0
:1017D000B7E0B7B9BEDB2ADC3FDCF2D8B3D94CDCCA
:1017E0008ADCD4DA2ADB2DDB99DB95FFB0E095FDAE
:1017F000B6E0B7B9B3DB1ADC2FDC06D93DDC9ADCE6
:10180000C5DA1BDB1EDB8ADB95FFB6E095FDB0E099
:10181000B7B99FDB0BDC20DC33D92EDCA0DCB6DAD9
:101820000CDB0FDB7BDBB7E0B7B998DBFFDB14DC4D
:1018300059D922DCB3DCAADA00DB03DB6FDB95FFCE
:10184000B0E095FDB6E0B7B984DB74FFB2E074FD9B
:10185000B1E0B7B9B6B1B068B064B6B9E7DBFCDBEC
:101860000BDCAEDC93DAE9DAECDAFDD957DB71FF99
:1018700020C067FD1EC0B0919500B0939200B09358
:101880009300B0919100B0939A00B1E0B0939B00A7
:1018900014E624E1B0916D00B11728F07D7F7460EB
:1018A00020936C0006C0B0918D00B13008F081CF5C
:1018B00035C072FF10C067FD0EC0B0916C00BA95C4
:1018C00011F47B7F72CFB0936C00B0918D00B1307A
:1018D00008F06FCF23C0B0919000B13058F0B091B4
:1018E0009500B0939300B0919100B0939A00B1E04D
:1018F000B0939B00B0919000BA3F80F4B92FBF71B4
:1019000021F4B0916600BB2349F0B091740000EF60
:1019100067FF01C000E6B01708F44BCFF89477DCFE
:101920008090B300B2E0B093B300BCDC8092B3000F
:10193000209261002092620020926300522C20923B
:1019400096007E7F78941FD762DCB92FBF7129F48F
:10195000B0916600BB2309F4AECDB091B900B130AF
:1019600008F0CCCD6BCEEDE0F0E023D0053A09F0E5
:101970001BC0EEE0F0E01DD00A3509F015C03AE0DA
:10198000ACEAB0E0E3E0F0E014D00D9331963A9584
:10199000D9F735E1A8EBB0E0EFE0F0E00AD00D9325
:1019A00031963A95D9F702C03DDC0AD0E4E2F0E086
:1019B0000895E199FECFEEBBFFBBE09A0DB3089509
:1019C0001ED03AE0ACEAB0E0E3E0F0E00D910FD0D9
:1019D00031963A95D9F735E1A8EBB0E0EFE0F0E0C9
:1019E0000D9105D031963A95D9F712D00895E19925
:1019F000FECF0DBBEEBBFFBBE29AE19A0895EDE08E
:101A0000F0E00FEFF4DFEEE0F0E00FEFF0DF08952D
:101A1000EDE0F0E005EAEBDFEEE0F0E00AE5E7DF1D
:101A200008953091A9000091AA00313011F400937B
:101A3000AC00323011F40093AD00333011F4009358
:101A4000AE00343011F40093C000353011F400932F
:101A5000AF00363011F40093B200373011F4009328
:101A6000BE00383011F40093C700393011F40093F0
:101A7000BF003A3011F40093B3003B3011F40093EF
:101A8000C8003C3011F40093B4003D3011F40093D1
:101A9000B500089525E081D62A95E9F7089588D6FE
:101AA0008AD68CD68ED673D683D685D687D689D657
:101AB0006ED67ED680D682D684D6089582D67ED63D
:101AC0007AD676D664D67DD679D675D671D65FD6D7
:101AD00078D674D670D66CD608958090A900909070
:101AE000AA0066D665D664D652D68A94D1F769D64E
:101AF0004ED69A94E1F70895F894D1DF7894CADF2E
:101B0000C9DFB1E0B093A900B1E0B093AA00209280
:101B1000AB00F894E2DF7894B5E06B2E70908D0006
:101B20003CD6B0918D007B16C9F7B13018F0BF3F9D
:101B300040F107C076DFF89443DFB1DFB8E0B1BD14
:101B4000A9DF6A9459F7B091AB00B395B093AB009D
:101B5000B33008F4DECF9EDFB091AA00B395B09306
:101B6000AA00F894B091A900BA95E6E4F0E0EB0F72
:101B7000F21D049178940395B091AA00B01708F46F
:101B8000C6CF88DF87DFB091A900B395B093A900D5
:101B9000B091A900BE3008F4B7CF44DBF89410DF51
:061BA000B8E0B1BD77DFE3
:00000001FF
